:020000040000FA
:060000003DEF2FF012009D
:062000003DEF2FF012007D
:06200800CAEF2BF01200EC
:06201800CAEF2BF01200DC
:02202A000000B4
:04202C00D9CFE6FF23
:10203000E1CFD9FFE652928092820D0EC16E030E5F
:10204000C06E9284809489949286809689969288B4
:102050008998899A929A938093828A9693968A888D
:102060009398938A818AF19E8A9493948B9094900A
:102070008B9294928B949494949C8B9CDF6A400EE8
:10208000DF5C10E2DF50EA6A010FE96E010EEA221E
:10209000EF6ADF50EA6A410FE96E010EEA22EF6A49
:1020A000DF2AEDD70101816B0101020E826F010170
:1020B000030E836F0101040E846F0101050E856F0D
:1020C0000101060E866F0101080E876F0101180ECF
:1020D000886F01010A0E896F0101090E8A6F0101E3
:1020E0000B0E8B6F0101110E8C6F01018D690101C7
:1020F0008E6901018F6901019069080ED56E040E89
:10210000CA6E4F0ECB6E0C0EBD6E1D0EBE6E010163
:10211000400EE16F01013E0EE26F01013C0EE36FE4
:1021200001017E0E986F01012D0E996F0101936BD5
:10213000300EBE6E070EB46EB56AF28CF28EC56AB2
:10214000C76A280EC66E1F0EC86EA3EC2BF0E552B0
:10215000E552E7CFD9FF1200D9CFE6FFE1CFD9FF93
:10216000080EE12601019A6B400EE66E010EE66E46
:10217000010EE66E54EC2BF0E552E552E5520008F4
:1021800002E3E0EF1FF0400E01019A5D02E3E0EF91
:102190001FF001019A51EA6A010FE96E010EEA226D
:1021A000EF50420A02E1BCEF1FF00F0A02E187EF95
:1021B0001FF03E0A02E121EF1FF0140A02E1EDEFE9
:1021C0001EF0130A02E1C2EF1EF0E00A02E1B1EFD5
:1021D0001EF0070A02E18DEF1EF0010A02E186EF10
:1021E0001EF0030A02E181EF1EF0010A02E179EF1D
:1021F0001EF0170A02E1A1EF1DF0030A02E1CDEF84
:102200001CF0060A02E10CEF1CF0070A02E176EF6F
:102210001BF0030A02E114EF1BF0070A02E13EEF94
:102220001AF0010A02E19BEF19F0D30A02E126EF4E
:1022300019F0670A02E153EF18F07A0A02E1F1EFB0
:1022400017F0200A02E185EF17F00A0A02E16EEFAB
:1022500017F0200A02E157EF17F0330A02E126EFE8
:1022600017F0200A02E1F5EF16F0520A02E1EFEF53
:1022700016F0600A02E1E9EF16F0200A02E1E3EF4E
:1022800016F00C0A02E1B4EF16F00A0A02E1AEEF12
:1022900016F0110A02E1A8EF16F0200A02E1A2EFFF
:1022A00016F0020A02E19CEF16F03F0A02E196EFF7
:1022B00016F01F0A02E190EF16F0260A02E176EF0F
:1022C00016F0660A02E134EF16F07F0A02E12EEF03
:1022D00016F0390A02E1E1EF15F0350A02E1BEEF2E
:1022E00015F0120A01E161D3200A01E19CD2590ADA
:1022F00001E17FD20F0A01E168D2010A01E14DD26A
:10230000050A01E1F8D1070A01E152D10D0A01E104
:1023100044D10B0A01E128D1430A3BE0400A02E024
:10232000DCEF1FF001019A2B0101090E416F010141
:10233000220E426F0101630E436F0101020E446FD2
:102340000101290E456F0101950E466F010EE66EE3
:1023500040EC2DF0E55200090CE0C0EC2DF001013D
:10236000416FC0EC2DF00101426FC0EC2DF0010176
:10237000436F04010CBF0BD0400EE66E410EE66EBB
:10238000010EE66E18EC2BF0E552E552E552DEEF59
:102390001FF001019A2B92849286AFEC2BF00B0E6A
:1023A000C16EA60EC06E01019A51EA6A010FE96E74
:1023B000010EEA22EF50070B01019F6F070E01018A
:1023C0009F1512E101019B6B400E01019B5D0BE229
:1023D00001019B51EA6A410FE96E010EEA22EF6AA0
:1023E00001019B2BF1D7AAD0070E01019F5D13E1DC
:1023F000140EDE6EDD6A0A0EF36E020EF3CFDBFF03
:10240000030EDB6A0101806B01017F6B01017E6BB2
:1024100001017D6B1FD001019F0508E0020E010143
:102420009F5D04E0040E01019F5D0AE1DE6ADD6A42
:10243000200EF36E020EF3CFDBFF030EDB6A0AD031
:10244000200EDE6EDD6A100EF36E020EF3CFDBFFA0
:10245000030EDB6A01019B6B01019D6B020EDBCF5A
:102460000BF0030EDBCF0CF001010B509D5D000E55
:102470000C5464E201019C6B01019FA11AD0090E6A
:10248000C26EC282C2B2FED701019B51EA6A410FFD
:10249000E96E010EEA22C3CFEFFF01019B29EA6A30
:1024A000410FE96E010EEA22C4CFEFFFDF500101B8
:1024B0009C2701019FA31ED00D0EC26EC282C2B224
:1024C000FED701019B5101019C25EA6A410FE96E8B
:1024D000010EEA22C3CFEFFF01019B2901019C25D8
:1024E000EA6A410FE96E010EEA22C4CFEFFFDF5026
:1024F00001019C2701019FA51BD0050EC26EC2825F
:10250000C2B2FED701019B5101019C25EA6A410F2D
:10251000E96E010EEA22C3CFEFFF01019B29010101
:102520009C25EA6A410FE96E010EEA22C4CFEFFF53
:10253000020E01019B2701019D2B90D704010CBFC6
:102540000BD0400EE66E410EE66E010EE66E18EC04
:102550002BF0E552E552E5520D0EC16E01019A2BAA
:10256000A3EC2BF0DEEF1FF001019B6B040E0101C9
:102570009B5D11E201019A51EA6A010FE96E010EB9
:10258000EA22EF50E66E40EC2DF0E55201019A2B65
:1025900001019B2BEBD7DEEF1FF001019A2B090EF7
:1025A000E66E40EC2DF0E552DEEF1FF0DEEF1FF09F
:1025B00001019A2B0101090E416F0101220E426FA8
:1025C0000101630E436F0101020E446F0101290EE8
:1025D000456F0101950E466F040EE66E40EC2DF03E
:1025E000E552000901E177D001019A519A2BEA6A7C
:1025F000010FE96E010EEA22EF50E66E40EC2DF07D
:10260000E55201019A519A2BEA6A010FE96E010E17
:10261000EA22EF50E66E40EC2DF0E55201019A29D6
:10262000EA6A010FE96E010EEA22EFCF0BF00C6AA5
:102630000BBE0C680BC0DEFF0CC0DDFFD9CFE9FF7D
:10264000DACFEAFFEE50ED6EEF6A01019A51EA6AC5
:10265000010FE96E010EEA22EFCF0BF00C6A0BBE00
:102660000C680BC0DEFF0CC0DDFF01019A519A2BF4
:10267000EA6A010FE96E010EEA22EF50E66E40ECC5
:102680002DF0E55201019A519A2BEA6A010FE96E89
:10269000010EEA22EF50E66E40EC2DF0E55201010A
:1026A0009B6BDECF0BF0DDCF0CF001010B509B5D7F
:1026B000000E0C5410E2C0EC2DF0E66E01019B51AF
:1026C000EA6A410FE96E010EEA22E552E750EF6E29
:1026D00001019B2BE6D704010CBF0BD0400EE66E28
:1026E000410EE66E010EE66E18EC2BF0E552E55257
:1026F000E552DEEF1FF0040E01019A25EA6A010F90
:10270000E96E010EEA22EFCF0BF00C6A0BBE0C68EB
:102710000BC0DEFF0CC0DDFFD9CFE9FFDACFEAFF47
:10272000EE50ED6EEF6A030E01019A25EA6A010F81
:10273000E96E010EEA22EFCF0BF00C6A0BBE0C68BB
:102740000BC0DEFF0CC0DDFF01019B6BDECF0BF089
:10275000DDCF0CF0050E0B26000E0C2201010B50F4
:102760009B5D000E0C5411E201019A5101019B2561
:10277000EA6A010FE96E010EEA22EF50E66E40ECC4
:102780002DF0E55201019B2BE1D7050E01019A279F
:10279000DF5001019A27DEEF1FF001019A2B92967C
:1027A00089960C0EE66E1FEC2FF0E5528986780EA6
:1027B000E66E1FEC2FF0E55289963C0EE66E1FEC9C
:1027C0002FF0E5529286DEEF1FF001019A2B0101F6
:1027D0009A51EA6A010FE96E010EEA22EF5003E115
:1027E0008A94898A02D0899A8A8401019A2BDEEF21
:1027F0001FF001019A2B80A604D00101010E416F48
:1028000002D00101416B04010CBF0BD0400EE66EFB
:10281000410EE66E010EE66E18EC2BF0E552E55225
:10282000E552DEEF1FF001019A2B030E01019A25FC
:10283000EA6A010FE96E010EEA22EF5015E0030E7D
:1028400001019A25EA6A010FE96E010EEA22EFCF33
:102850000BF0400EE76E0B18E8AE02D00B3403D03D
:10286000E750D8800B5405E2040E01019A27DEEFF1
:102870001FF0020E01019A25EA6A010FE96E010EAE
:10288000EA22EF50010B5009E82401019E6FC58038
:10289000C5B0FED79E969EC1C9FF9EA6FED7C5AC09
:1028A0000FD0C584030E01019A25EA6A010FE96E73
:1028B000010EEA22EF50040F01019A27DEEF1FF00C
:1028C0009E9601019A29EA6A010FE96E010EEA2239
:1028D000EF50C96E9EA6FED7C5AC0FD0C584030EBF
:1028E00001019A25EA6A010FE96E010EEA22EF5012
:1028F000040F01019A27DEEF1FF09E9601019A5105
:10290000EA6A010FE96E010EEA22EF50C96E9EA637
:10291000FED7C5AC0FD0C584030E01019A25EA6A23
:10292000010FE96E010EEA22EF50040F01019A2710
:10293000DEEF1FF0030E01019A25EA6A010FE96E2E
:10294000010EEA22EFCF9DF1040E01019A27010149
:102950009B6B9E9601019A519A2BEA6A010FE96ED0
:10296000010EEA22EF50C96E9EA6FED7C5AC0ED06E
:10297000C584030E01019A25EA6A010FE96E010E72
:10298000EA22EF50040F01019A2707D001019B2B87
:1029900001019D5101019B5DDCE3C584060EE66EDD
:1029A00008EC2FF0E552DEEF1FF001019A2B030E29
:1029B00001019A25EA6A010FE96E010EEA22EF5041
:1029C00015E0030E01019A25EA6A010FE96E010E76
:1029D000EA22EFCF0BF0400EE76E0B18E8AE02D004
:1029E0000B3403D0E750D8800B5405E2040E0101EC
:1029F0009A27DEEF1FF0020E01019A25EA6A010F05
:102A0000E96E010EEA22EF50010B5009E8240101A2
:102A10009E6FC580C5B0FED79E969EC1C9FF9EA67B
:102A2000FED7C5AC0FD0C584030E01019A25EA6A12
:102A3000010FE96E010EEA22EF50040F01019A27FF
:102A4000DEEF1FF09E9601019A29EA6A010FE96EF6
:102A5000010EEA22EF50C96E9EA6FED7C5AC0FD07C
:102A6000C584030E01019A25EA6A010FE96E010E81
:102A7000EA22EF50040F01019A27DEEF1FF09E9625
:102A800001019A51EA6A010FE96E010EEA22EF5044
:102A9000C96E9EA6FED7C5AC0FD0C584030E01013A
:102AA0009A25EA6A010FE96E010EEA22EF50040F3F
:102AB00001019A27DEEF1FF0C582C5B2FED79E96B0
:102AC000010E01019E11C96E9EA6FED7C5AC0FD0A6
:102AD000C584030E01019A25EA6A010FE96E010E11
:102AE000EA22EF50040F01019A27DEEF1FF0030ED8
:102AF00001019A25EA6A010FE96E010EEA22EFCF81
:102B00009DF101019B6B9E96C5869EA6FED7010195
:102B10009B519B2BEA6A410FE96E010EEA22C9CF55
:102B2000EFFF01019D5101019B5D02E1C58A01D0CA
:102B3000C59AC588C5B8FED701019D5101019B5DAD
:102B4000E2E3030E01019A25EA6A010FE96E010E24
:102B5000EA22EF50040F01019A27C58404010CBF3B
:102B60000BD0400EE66E410EE66E010EE66E18ECDE
:102B70002BF0E552E552E552DEEF1FF002C181F184
:102B800003C182F104C183F105C184F106C185F15D
:102B900007C186F108C187F109C188F10AC189F12D
:102BA0000BC18AF10CC18BF10DC18CF10EC18DF1FD
:102BB0000FC18EF110C18FF10101400E9A6FDEEF4F
:102BC0001FF001019A2B01019A51EA6A010FE96E87
:102BD000010EEA22EF50040B1FE0ECEC1FF0050E93
:102BE000C26E780EE66E08EC2FF0E552C282C2B2D9
:102BF000FED79E9CC3CF41F1C4CF42F104010CBF6C
:102C00000BD0400EE66E410EE66E010EE66E18EC3D
:102C10002BF0E552E552E55201019A51EA6A010FA3
:102C2000E96E010EEA22EF50010B03E0EFEC1FF01A
:102C300002D0ECEC1FF001019A51EA6A010FE96E33
:102C4000010EEA22EF50020B03E023EC27F002D042
:102C500027EC27F001019A2BDEEF1FF001019A2BE0
:102C600040EC20F0DEEF1FF001019A2B58EC20F031
:102C7000DEEF1FF001019A51EA6A010FE96E010EC1
:102C8000EA22EF50040B1FE0ECEC1FF0050EC26EC1
:102C9000780EE66E08EC2FF0E552C282C2B2FED783
:102CA0009E9CC3CF41F1C4CF42F104010CBF0BD0B5
:102CB000400EE66E410EE66E010EE66E18EC2BF04D
:102CC000E552E552E55201019A51EA6A010FE96EB7
:102CD000010EEA22EF50020B03E023EC27F002D0B2
:102CE00027EC27F001019A2BDEEF1FF00101010E06
:102CF000416F0101150E426F0101436B04010CBFCE
:102D00000BD0400EE66E410EE66E010EE66E18EC3C
:102D10002BF0E552E552E55201019A2BDEEF1FF050
:102D2000F2EC1FF001019A2BDEEF1FF00EEC20F009
:102D300001019A2BDEEF1FF02CEC20F001019A2B01
:102D4000DEEF1FF0F5EC21F001019A2BDEEF1FF012
:102D50002EEC22F001019A2BDEEF1FF08EEC22F018
:102D600001019A2BDEEF1FF001019A29EA6A010F97
:102D7000E96E010EEA22EF50DE6EDD6A020E0101FD
:102D80009A25EA6A010FE96E010EEA22EFCF0BF0F5
:102D90000C6A0BBE0C680BC00CF00B6AD9CFE9FFB4
:102DA000DACFEAFF0B50EE260C50ED22DECFE6FF25
:102DB000DDCFE6FFC9EC21F0E552E552030E01013B
:102DC0009A27DEEF1FF099EC22F001019A2BDEEF3B
:102DD0001FF0A3EC22F001019A2BDEEF1FF0ADEC07
:102DE00022F001019A2BDEEF1FF001019A29EA6A15
:102DF000010FE96E010EEA22EF50DE6EDD6A020E6F
:102E000001019A25EA6A010FE96E010EEA22EFCF6D
:102E10000DF00E6A0DBE0E680DC00EF00D6ADE508C
:102E20000D240B6EDD500E200C6E0BC0DEFF0CC0AF
:102E3000DDFFDECFE6FFDDCFE6FF14EC23F0E55249
:102E4000E552030E01019A27DEEF1FF001019A29D6
:102E5000EA6A010FE96E010EEA22EF50DE6EDD6ACA
:102E6000020E01019A25EA6A010FE96E010EEA22BB
:102E7000EFCF0DF00E6A0DBE0E680DC00EF00D6A9C
:102E8000DE500D240B6EDD500E200C6E0BC0DEFFED
:102E90000CC0DDFFDECFE6FFDDCFE6FF2EEC23F03A
:102EA000E552E552030E01019A27DEEF1FF0010102
:102EB0009A29EA6A010FE96E010EEA22EF50DE6EEE
:102EC000DD6ADECFE6FFDDCFE6FFD5EC22F0E5528E
:102ED000E552020E01019A27DEEF1FF001019A2947
:102EE000EA6A010FE96E010EEA22EF50DE6EDD6A3A
:102EF000DECFE6FFDDCFE6FFF4EC22F0E552E5524F
:102F0000020E01019A27DEEF1FF001019A2B010149
:102F10009A519A2BEA6A010FE96E010EEA22EFCF6D
:102F20009DF101019B6B01019D5101019B5D3CE203
:102F300001019B5105E086C1E6FF66EC20F0E552F9
:102F400001019A29EA6A010FE96E010EEA22EF50A7
:102F50003F0B0B6E0C6A0BBE0C680BC0DEFF0CC087
:102F6000DDFFD9CFE9FFDACFEAFFEE50ED6EEF6A71
:102F700001019A51EA6A010FE96E010EEA22EF504F
:102F8000DF1282C1E6FF66EC20F0E552DECFE6FFFD
:102F9000DDCFE6FF8CEC20F0E552E552020E010198
:102FA0009A2701019B2BBFD788C1E6FF66EC20F072
:102FB000E552030EE66E08EC2FF0E55289C1E6FFFC
:102FC00066EC20F0E5520C0EE66E2FEC2FF0E55289
:102FD00086C1E6FF66EC20F0E552A3EC2CF0DEEFB4
:102FE0001FF001019A2B01019A519A2BEA6A010FF5
:102FF000E96E010EEA22EFCF9DF101019B6B010109
:103000009D5101019B5D3CE201019B5105E086C1A0
:10301000E6FF66EC20F0E55201019A29EA6A010F09
:10302000E96E010EEA22EF503F0B0B6E0C6A0BBEED
:103030000C680BC0DEFF0CC0DDFFD9CFE9FFDACF93
:10304000EAFFEE50ED6EEF6A01019A51EA6A010F54
:10305000E96E010EEA22EF50DF1282C1E6FF66EC54
:1030600020F0E552DECFE6FFDDCFE6FF8CEC20F06E
:10307000E552E552020E01019A2701019B2BBFD7B1
:1030800087C1E6FF66EC20F0E5520A0EE66E08EC1A
:103090002FF0E55286C1E6FF66EC20F0E552A3EC86
:1030A0002CF0DEEF1FF0020E01019A25EA6A010FF3
:1030B000E96E010EEA22EF503F0B0B6E0C6A0BBE5D
:1030C0000C680BC0DEFF0CC0DDFFD9CFE9FFDACF03
:1030D000EAFFEE50ED6EEF6A01019A29EA6A010FEC
:1030E000E96E010EEA22EF50DF12040E01019A256B
:1030F000EA6A010FE96E010EEA22EF503F0B0B6EF8
:103100000C6A0BBE0C68020E0BC0DBFF030E0CC07A
:10311000DBFFD950020FE96EDACFEAFFEE50ED6E19
:10312000EF6A030E01019A25EA6A010FE96E010EAA
:10313000EA22EF500B6E0C6AD950020FE96EDACF1B
:10314000EAFF0B50EE120C50ED12060E01019A250B
:10315000EA6A010FE96E010EEA22EF503F0B0B6E97
:103160000C6A0BBE0C68040E0BC0DBFF050E0CC016
:10317000DBFFD950040FE96EDACFEAFFEE50ED6EB7
:10318000EF6A050E01019A25EA6A010FE96E010E48
:10319000EA22EF500B6E0C6AD950040FE96EDACFB9
:1031A000EAFF0B50EE120C50ED12080E01019A25A9
:1031B000EA6A010FE96E010EEA22EF503F0B0B6E37
:1031C0000C6A0BBE0C68060E0BC0DBFF070E0CC0B2
:1031D000DBFFD950060FE96EDACFEAFFEE50ED6E55
:1031E000EF6A070E01019A25EA6A010FE96E010EE6
:1031F000EA22EF500B6E0C6AD950060FE96EDACF57
:10320000EAFF0B50EE120C50ED12060EDBCFE6FF7C
:10321000070EDBCFE6FF040EDBCFE6FF050EDBCFAC
:10322000E6FF020EDBCFE6FF030EDBCFE6FFDECFCD
:10323000E6FFDDCFE6FF49EC23F0F56E080EE15E18
:10324000F550090E01019A27DEEF1FF001019A29BE
:10325000EA6A010FE96E010EEA22EF50DE6EDD6AC6
:10326000020E01019A25EA6A010FE96E010EEA22B7
:10327000EFCF0DF00E6A0DBE0E680DC00EF00D6A98
:10328000DE500D240B6EDD500E200C6E0BC0DEFFE9
:103290000CC0DDFF020EDBCFE6FF030EDBCFE6FF47
:1032A000DECFE6FFDDCFE6FFAAEC26F0E552E552E1
:1032B000E552E552040EF3CFDBFF050EF4CFDBFF42
:1032C000FF0EE76E040EDBCF0BF0050EDBCF0CF02C
:1032D000E7500B160C6A0BC041F1D950040FE96E90
:1032E000DACFEAFF080E0F0B06E0EC52D890ED3271
:1032F000EF32E806FAE1FF0EE76E040EDBCF0BF0CB
:10330000050EDBCF0CF0E7500B160C6A0BC042F138
:1033100004010CBF0BD0400EE66E410EE66E010EAE
:10332000E66E18EC2BF0E552E552E552050E010170
:103330009A27DEEF1FF001019A2B01019A519A2B77
:10334000EA6A010FE96E010EEA22EFCF9DF1010159
:103350009A519A2BEA6A010FE96E010EEA22EF50A8
:10336000E66E0E0EE66EE66A96EC23F0E552E55246
:10337000E552F60EE66E6E0EE66EE66A96EC23F009
:10338000E552E552E55201019A519A2BEA6A010F82
:10339000E96E010EEA22EF50E66E0E0EE66EE66A68
:1033A00096EC23F0E552E552E552F70EE66E6E0E0E
:1033B000E66EE66A96EC23F0E552E552E55201012D
:1033C0009A519A2BEA6A010FE96E010EEA22EF5038
:1033D000E66E0E0EE66EE66A96EC23F0E552E552D6
:1033E000E552F80EE66E6E0EE66EE66A96EC23F097
:1033F000E552E552E552080EE66EFCEC23F0E5528C
:10340000ECEC20F0F3CFDEFFF4CFDDFF01019B6B8E
:1034100001019D5101019B5D1FE2090EE66EFCEC6E
:1034200023F0E552ECEC20F0F3CFDEFFF4CFDDFF2C
:10343000DECF0BF0DDCF0CF0FF0E0B16000E0C16DE
:1034400001019B51EA6A410FE96E010EEA220BC0AD
:10345000EFFF01019B2BDCD704010CBFFDD7400E11
:10346000E66E410EE66E010EE66E18EC2BF0E552AC
:10347000E552E552A3EC2CF0DEEF1FF001019A2B90
:1034800001019A519A2BEA6A010FE96E010EEA22B4
:10349000EFCF9DF101019A519A2BEA6A010FE96E73
:1034A000010EEA22EFCF0BF00C6A0BBE0C680BC0CA
:1034B000DEFF0CC0DDFF01019A519A2BEA6A010F71
:1034C000E96E010EEA22EFCF0BF00C6A0BBE0C681E
:1034D000020E0BC0DBFF030E0CC0DBFFA60EE66E78
:1034E0009E0EE66EE66A96EC23F0E552E552E55252
:1034F000A60EE66E9C0EE66EE66A96EC23F0E552AA
:10350000E552E552020EDBCFE6FF0E0EE66EE66AEE
:1035100096EC23F0E552E552E552AA0EE66E6E0EE9
:10352000E66EE66A96EC23F0E552E552E5520101BB
:103530009B6B01019D5101019B5D64E2DFCFE6FFC2
:103540000E0EE66EE66A96EC23F0E552E552E55281
:10355000A90EE66E6E0EE66EE66A96EC23F0E55274
:10356000E552E552A60EE66E800EE66EE66A96EC31
:1035700023F0E552E552E552A80EE66E500EE66ED7
:10358000E66A96EC23F0E552E552E552F50EE66E5A
:103590006E0EE66EE66A96EC23F0E552E552E552D1
:1035A000A90EE66E6E0EE66EE66A96EC23F0E55224
:1035B000E552E552020EE66EFCEC23F0E552ECEC2F
:1035C00020F0060EF3CFDBFF070EF4CFDBFFFF0E7C
:1035D000E76E060EDBCF0BF0070EDBCF0CF0E750EB
:1035E0000B160C6A01019B51EA6A410FE96E010E4C
:1035F000EA220BC0EFFFDF2A010E01E3DB2A010103
:103600009B2B97D704010CBFFDD7400EE66E410EF1
:10361000E66E010EE66E18EC2BF0E552E552E5522F
:10362000A3EC2CF0DEEF1FF001019A2B040EE66EE6
:103630000E0EE66EE66A96EC23F0E552E552E55290
:10364000F60EE66E6E0EE66EE66A96EC23F0E55236
:10365000E552E552E66A0E0EE66EE66A96EC23F057
:10366000E552E552E552F70EE66E6E0EE66EE66A3C
:1036700096EC23F0E552E552E5523C0EE66E0E0E56
:10368000E66EE66A96EC23F0E552E552E552F80E56
:10369000E66E6E0EE66EE66A96EC23F0E552E552B3
:1036A000E55201019A519A2BEA6A010FE96E010E67
:1036B000EA22EFCF9DF19DC1E6FFE66A0C0EE66EB1
:1036C00096EC23F0E552E552E552E66AE66AE66AD0
:1036D00096EC23F0E552E552E55258EC24F0FA0E50
:1036E000E66E08EC2FF0E552DEEF1FF001019A2B99
:1036F000050EE66E0E0EE66EE66A96EC23F0E552D7
:10370000E552E552F60EE66E6E0EE66EE66A96EC51
:1037100023F0E552E552E552E66A0E0EE66EE66AE1
:1037200096EC23F0E552E552E552F70EE66E6E0E8A
:10373000E66EE66A96EC23F0E552E552E5523C0E61
:10374000E66E0E0EE66EE66A96EC23F0E552E55262
:10375000E552F80EE66E6E0EE66EE66A96EC23F023
:10376000E552E552E55201019A29EA6A010FE96E34
:10377000010EEA22EFCF9DF19DC1E6FF9DC1E6FF5C
:103780000C0EE66E96EC23F0E552E552E552E66A41
:10379000E66AE66A96EC23F0E552E552E552040E3D
:1037A000E66E0E0EE66EE66A96EC23F0E552E55202
:1037B000E552F60EE66E6E0EE66EE66A96EC23F0C5
:1037C000E552E552E55201019A51EA6A010FE96EAC
:1037D000010EEA22EFCF9DF19DC1E6FF9DC1E6FFFC
:1037E0000C0EE66E96EC23F0E552E552E552E66AE1
:1037F000E66AE66A96EC23F0E552E552E55258ECAB
:1038000024F0C80EE66E08EC2FF0E552020E01011E
:103810009A27A3EC2CF0D2D3A60EE66E8E0EE66E9F
:10382000E66A96EC23F0E552E552E552A60EE66E06
:103830009C0EE66EE66A96EC23F0E552E552E55200
:10384000020E01019A25EA6A010FE96E010EEA22D1
:10385000EF50E66E0E0EE66EE66A96EC23F0E55249
:10386000E552E552F60EE66E6E0EE66EE66A96ECF0
:1038700023F0E552E552E552030E01019A25EA6A6A
:10388000010FE96E010EEA22EF50E66E0E0EE66EB3
:10389000E66A96EC23F0E552E552E552F70EE66E45
:1038A0006E0EE66EE66A96EC23F0E552E552E552BE
:1038B000040E01019A25EA6A010FE96E010EEA225F
:1038C000EF50E66E0E0EE66EE66A96EC23F0E552D9
:1038D000E552E552F80EE66E6E0EE66EE66A96EC7E
:1038E00023F0E552E552E55201019A29EA6A010FF7
:1038F000E96E010EEA22EFCF9DF1050E01019A2734
:1039000001019B6B01019D0501019B5D22E201010B
:103910009A519A2BEA6A010FE96E010EEA22EFCF63
:103920009FF101019A519A2BEA6A010FE96E010E8B
:10393000EA22EFCF9EF19FC1E6FF9EC1E6FF0D0E8A
:10394000E66E96EC23F0E552E552E55201019B2B21
:10395000D9D701019A519A2BEA6A010FE96E010E3B
:10396000EA22EFCF9FF101019A519A2BEA6A010FE7
:10397000E96E010EEA22EFCF9EF19FC1E6FF9EC1E4
:10398000E6FF0F0EE66E96EC23F0E552E552E552A7
:1039900026EC24F0A3EC2CF011D3A60EE66E8E0ECE
:1039A000E66EE66A96EC23F0E552E552E552A60E85
:1039B000E66E8C0EE66EE66A96EC23F0E552E55272
:1039C000E552A60EE66E840EE66EE66A96EC23F0ED
:1039D000E552E552E552E66AEF0EE66EE66A96ECCF
:1039E00023F0E552E552E552E66AF80EE66EE66A25
:1039F00096EC23F0E552E552E552300EE66E0E0EDF
:103A0000E66EE66A96EC23F0E552E552E552F80ED2
:103A1000E66E6E0EE66EE66A96EC23F0E552E5522F
:103A2000E552E66A0E0EE66EE66A96EC23F0E55283
:103A3000E552E552F70EE66E6E0EE66EE66A96EC1D
:103A400023F0E552E552E55201019A2B01019A510A
:103A50009A2BEA6A010FE96E010EEA22EFCF9BF181
:103A60009BC1E6FF0E0EE66EE66A96EC23F0E55289
:103A7000E552E552F60EE66E6E0EE66EE66A96ECDE
:103A800023F0E552E552E55201019A519A2BEA6A78
:103A9000010FE96E010EEA22EFCF9FF101019A5169
:103AA0009A2BEA6A010FE96E010EEA22EFCF9EF12E
:103AB0009FC1E6FF9EC1E6FF0F0EE66E96EC23F077
:103AC000E552E552E55226EC24F001019B2B9BC107
:103AD000E6FF0E0EE66EE66A96EC23F0E552E5523E
:103AE000E552F60EE66E6E0EE66EE66A96EC23F092
:103AF000E552E552E5529FC1E6FF9EC1E6FF0F0E7B
:103B0000E66E96EC23F0E552E552E55226EC24F001
:103B1000E66AE66AE66A96EC23F0E552E552E5527B
:103B2000E66AE66AE66A96EC23F0E552E552E5526B
:103B3000E66AE66AE66A96EC23F0E552E552E5525B
:103B40003DD2A60EE66E9E0EE66EE66A96EC23F079
:103B5000E552E552E552A60EE66E9C0EE66EE66A6A
:103B600096EC23F0E552E552E552A60EE66E840E81
:103B7000E66EE66A96EC23F0E552E552E552010165
:103B80009A29EA6A010FE96E010EEA22EFCF9DF150
:103B9000020E01019A25EA6A010FE96E010EEA227E
:103BA000EFCF9FF1030E01019A25EA6A010FE96E3A
:103BB000010EEA22EFCF9EF1040E01019A270101C6
:103BC0009B6B01019D5101019B5D01E385D09FC16C
:103BD000E6FF0E0EE66EE66A96EC23F0E552E5523D
:103BE000E552A90EE66E6E0EE66EE66A96EC23F0DE
:103BF000E552E552E5529EC1E6FF0E0EE66EE66A1C
:103C000096EC23F0E552E552E552AA0EE66E6E0EF2
:103C1000E66EE66A96EC23F0E552E552E5520101C4
:103C20009A519A2BEA6A010FE96E010EEA22EF50CF
:103C3000E66E0E0EE66EE66A96EC23F0E552E5526D
:103C4000E552A80EE66E6E0EE66EE66A96EC23F07E
:103C5000E552E552E552550EE66E0E0EE66EE66A48
:103C600096EC23F0E552E552E552A70EE66E6E0E95
:103C7000E66EE66A96EC23F0E552E552E552AA0EAE
:103C8000E66E0E0EE66EE66A96EC23F0E552E5521D
:103C9000E552A70EE66E6E0EE66EE66A96EC23F02F
:103CA000E552E552E552A60EE66E820EE66EE66A33
:103CB00096EC23F0E552E552E552E66AE66AE66ADA
:103CC00096EC23F0E552E552E55258EC24F0010160
:103CD0009F2B01019B2B75D7A60EE66E940EE66E08
:103CE000E66A96EC23F0E552E552E552A3EC2CF09F
:103CF00065D1A1EC2BF08B9285EC24F001019A2B7D
:103D00005DD1E1EC24F001019A2B58D1F1EC24F0C3
:103D100001019A2BA3EC2CF051D101019A2B010146
:103D20009B6B200E01019B5D18E201019A5101017C
:103D30009B25EA6A010FE96E010EEA22EF50E66E5A
:103D400001019B51EA6AA00FE96E010EEA22E552D9
:103D5000E750EF6E01019B2BE4D7200E01019A275B
:103D60002DD101019A2B9AC1E6FFA00EE66E010E3D
:103D7000E66E87EC25F0E552E552E552230E01018F
:103D80009A271CD1929689969294899401019A2B34
:103D900001019A51EA6A010FE96E010EEA22EFCFA2
:103DA0009DF101019B6B01019D5101019B5D10E2A1
:103DB00001019A2B01019A51EA6A010FE96E010E85
:103DC000EA22EF50E66EDAD9E55201019B2BEBD7E0
:103DD0009286928401019A2BF1D0F29E01019A2BD6
:103DE00001019A51EA6A010FE96E010EEA22EFCF52
:103DF0009DF101019B6B01019D5101019B5D0FE252
:103E00005EDAE66E01019B51EA6A410FE96E010E2E
:103E1000EA22E552E750EF6E01019B2BECD7F28EC0
:103E200004010CBF0BD0400EE66E410EE66E010E93
:103E3000E66E18EC2BF0E552E552E55201019A2BA3
:103E4000BDD0020E01019A25EA6A010FE96E010E4A
:103E5000EA22EF50BE6E01019A29EA6A010FE96E6B
:103E6000010EEA22EF50E840E8403F0B0B6E0C6A6F
:103E70000BBE0C680BC0DEFF0CC0DDFF300EDE1683
:103E8000DD6ACF0EBD14BD6EBD500D6E0E6ADE50E4
:103E90000D100B6EDD500E100C6E0B50BD6E030E30
:103EA00001019A25EA6A010FE96E010EEA22EFCFBD
:103EB000E1F1040E01019A25EA6A010FE96E010E93
:103EC000EA22EF280101E26F040E01019A25EA6A55
:103ED000010FE96E010EEA22EF040101E36F050E06
:103EE00001019A25EA6A010FE96E010EEA22EFCF7D
:103EF00098F1060E01019A25EA6A010FE96E010E9A
:103F0000EA22EFCF99F1070E01019A2757D081A637
:103F100002D00101938181B802D00101938381A471
:103F200002D0010193859D50400B05E0C250020B69
:103F300002E00101938B93C141F19D9C94C142F138
:103F400095C143F196C144F197C145F19D8C0101A2
:103F5000936BB9EC2BF004010CBF0BD0400EE66E56
:103F6000410EE66E010EE66E18EC2BF0E552E552BE
:103F7000E55201019A2B22D0A1EC2CF0840EA66E02
:103F8000FE0EF66E7F0EF76EF86AF56A0C00550E9F
:103F9000A76EAA0EA76EA6820101916B926B01011A
:103FA0009107000E925B01019151921103E0000014
:103FB0000000F5D7FF0002D001019A2BC3EF10F0EB
:103FC000F56E080EE15C02E2E16AE552E16EF55041
:103FD000E552E7CFD9FF12008A888A8612008A96B6
:103FE0008A9812008B80898A8A949DEC2BF0929695
:103FF000899692948994780EE66E08EC2FF0E5523B
:10400000899A8A84120EE66E49EC2FF0E552E7DFBA
:10401000010EE66E08EC2FF0E55212008B80898AC3
:104020008A949DEC2BF08996929689968994929425
:104030008994780EE66E08EC2FF0E552D0DF120E70
:10404000E66E49EC2FF0E552899A8A84010EE66EFD
:1040500008EC2FF0E5521200BFDF780EE66E49EC57
:104060002FF0E5528A94898A0C0EE66E08EC2FF048
:10407000E552899AA1EC2BF0928692848B901200E3
:104080008B80898A8A949DEC2BF0899692968996EA
:10409000899492948994780EE66E08EC2FF0E5529C
:1040A000899A8A84010EE66E08EC2FF0E552120020
:1040B0008A94898A0C0EE66E08EC2FF0E552899AF4
:1040C000A1EC2BF0928692848B901200D9CFE6FF60
:1040D000E1CFD9FFE65292948996DF6A060EDF5C43
:1040E00014E2FE0EDB50010BE8B08984E8A089944D
:1040F00000008986FE0EDBCFF3FFF390F342FE0E45
:10410000F3CFDBFF8996DF2AE9D789949284E552C1
:10411000E552E7CFD9FF1200D9CFE6FFE1CFD9FFB3
:10412000E6529294FD0EDBCFC0F1FE0EDBCFC1F163
:104130008986DF6A0E0EDF5C10E289960101C051AC
:10414000010B02E0898401D0899400008986D8900F
:104150000101C133C033DF2AEDD78996000000008A
:104160008986000000008996020EE66E49EC2FF069
:10417000E552E552E552E7CFD9FF1200D9CFE6FF6D
:10418000E1CFD9FFE652FE0EDBCFC2F1DF6A080EA7
:10419000DF5C17E289960C0EE66E2FEC2FF0E552ED
:1041A0000101C2A102D0898401D0899489860C0EB4
:1041B000E66E2FEC2FF0E5520101C291C243DF2AD7
:1041C000E6D789960C0EE66E2FEC2FF0E552E552FD
:1041D000E552E7CFD9FF1200D9CFE6FFE1CFD9FFF3
:1041E000E652DF6A080EDF5C0AE289860000000002
:1041F00000008996000000000000DF2AF3D79284B7
:104200000101C36BC46BDF6A080EDF5C14E28986B0
:10421000000000000000D8900101C433C33380A423
:1042200002D00101C38F0000899600000000000049
:104230000000DF2AE9D79294020EE66E49EC2FF0D7
:10424000E552C3C1F3FFC4C1F4FF00D0E552E5520B
:10425000E7CFD9FF1200D9CFE6FFE1CFD9FFE65271
:1042600092840101C56BC66B8986000000008996A7
:10427000DF6A0E0EDF5C10E289860000000000009D
:1042800080A402D00101C68D00008996D89001015A
:10429000C633C533DF2AEDD7898600000000899632
:1042A000020EE66E49EC2FF0E552C5C1F3FFC6C120
:1042B000F4FF00D0E552E552E7CFD9FF1200D9CF85
:1042C000E6FFE1CFD9FF020EE1260101C76BC86B03
:1042D000DF6A080EDF5C4EE2010EDB6A010EDB5086
:1042E0000B6E0C6AD8900C5004E6FA0E0B5C000EB4
:1042F0000C5809E280A604D0DE52FB0EDD6E02D01F
:10430000010EDB2AEBD7010EDB500B6E0C6AFA0EA6
:104310000B1801E10C5002E1550E2FD0010EDB6AA3
:10432000010EDB500B6E0C6AD8900C5004E6FA0EAE
:104330000B5C000E0C5809E280B604D0DE52FB0E76
:10434000DD6E02D0010EDB2AEBD7010EDB500B6EC7
:104350000C6AFA0E0B1801E10C5002E1AA0E0DD006
:1043600080A402D00101C881D8900101C833C733AD
:10437000DF2AAFD70101C75100D0F56E020EE15C14
:1043800002E2E16AE552E16EF550E552E7CFD9FF6E
:104390001200D9CFE6FFE1CFD9FF020EE126DE6A97
:1043A000DD6ADECF0BF0DDCF0CF0FD0EDBCF0DF0C4
:1043B000FE0EDBCF0EF00D500B5C0E500C5809E2D8
:1043C00086C1E6FF83DEE552DF2A010E01E3DB2A28
:1043D000E8D7F56E020EE15C02E2E16AE552E16EB9
:1043E000F550E552E7CFD9FF1200D9CFE6FFE1CF74
:1043F000D9FFE652DF6A400EDF5C1BE285C1E6FFB3
:1044000065DEE55228DFF3CF0BF0F4CF0CF0FF0EA2
:104410000B16000E0C16DF50EA6A410FE96E010E12
:10442000EA220BC0EFFF86C1E6FF50DEE552DF2A2D
:10443000E2D704010CBFFDD7400EE66E410EE66EDA
:10444000010EE66E18EC2BF0E552E552E552A3ECB6
:104450002CF0E552E552E7CFD9FF1200D9CFE6FFA5
:10446000E1CFD9FF030EE126DF6A400EDF5C3AE2BE
:1044700084C1E6FF2BDEE552EEDEDE52F3CFDEFF37
:10448000F4CFDDFFDD52FF0EE76E010EDBCF0BF048
:10449000020EDBCF0CF0E7500B160C6ADF50DF2A60
:1044A000EA6A410FE96E010EEA220BC0EFFF010E2E
:1044B000DBCF0BF0020EDBCF0CF00CC00BF00C6A64
:1044C000FF0E0B16000E0C16DF50EA6A410FE96E64
:1044D000010EEA220BC0EFFF86C1E6FFF7DDE552D1
:1044E000DF2AC3D704010CBFFDD7400EE66E410E94
:1044F000E66E010EE66E18EC2BF0E552E552E55241
:10450000A3EC2CF0F56E030EE15C02E2E16AE552E9
:10451000E16EF550E552E7CFD9FF120081C1E6FF09
:10452000D5DDE552000EE66EE66AF6DDE552E552AF
:1045300012008AC1E6FFCADDE5520C0EE66E08ECF9
:104540002FF0E55212008BC1E6FFC0DDE5520C0EE4
:10455000E66E08EC2FF0E55212008CC1E6FFB6DDE6
:10456000E5520C0EE66E08EC2FF0E552120087C102
:10457000E6FFACDDE552030EE66E08EC2FF0E552E7
:10458000120088C1E6FFA2DDE552030EE66E08ECDC
:104590002FF0E552120089C1E6FF98DDE5520C0EBE
:1045A000E66E2FEC2FF0E5521200D9CFE6FFE1CFF7
:1045B000D9FF83C1E6FF8ADDE552FD0EDBCFE6FFC2
:1045C000FE0EDBCFE6FFA8DDE552E552D0DF050E9B
:1045D000E66E08EC2FF0E55286C1E6FF77DDE55286
:1045E000E552E7CFD9FF1200D9CFE6FFE1CFD9FFDF
:1045F00083C1E6FF6BDDE552FD0EDBCFE6FFFE0E6D
:10460000DBCFE6FF89DDE552E552BBDF050EE66E46
:1046100008EC2FF0E552BFDF86C1E6FF57DDE5521B
:10462000E552E7CFD9FF1200D9CFE6FFE1CFD9FF9E
:1046300082C1E6FF4BDDE552FD0EDBCFE6FFFE0E4D
:10464000DBCFE6FF69DDE552E55291DF86C1E6FF8B
:104650003DDDE552E552E7CFD9FF1200D9CFE6FFA5
:10466000E1CFD9FF82C1E6FF31DDE552FD0EDBCFA0
:10467000E6FFFE0EDBCFE6FF4FDDE552E55281DFC0
:104680008ADF86C1E6FF22DDE552E552E7CFD9FF9A
:104690001200D9CFE6FFE1CFD9FF82C1E6FF16DDD8
:1046A000E552FD0EDBCFE6FFFE0EDBCFE6FF34DD8D
:1046B000E552E55286C1E6FF09DDE55282C1E6FF1B
:1046C00005DDE552FB0EDBCFE6FFFC0EDBCFE6FFA0
:1046D00023DDE552E55286C1E6FFF8DCE55282C1F2
:1046E000E6FFF4DCE552F90EDBCFE6FFFA0EDBCF96
:1046F000E6FF12DDE552E55286C1E6FFE7DCE55252
:1047000082C1E6FFE3DCE552F70EDBCFE6FFF80EF1
:10471000DBCFE6FF01DDE552E55229DF86C1E6FF8A
:10472000D5DCE552E552E7CFD9FF1200D9CFE6FF3D
:10473000E1CFD9FFE652FE0EDB500101C96FCA6B13
:10474000DF6A040EDF5C15E28996000000000000BD
:104750000101C951010B02E0898401D08994000054
:10476000000089860000D8900101CA33C933DF2ACE
:10477000E8D7FC0EDB500101C96FCA6BDF6A080E77
:10478000DF5C15E289960000000000000101C951BC
:10479000010B02E0898401D0899400000000898621
:1047A0000000D8900101CA33C933DF2AE8D7FD0ED3
:1047B000DB500101C96FCA6BDF6A080EDF5C15E2CE
:1047C00089960000000000000101C951010B02E0C0
:1047D000898401D089940000000089860000D89067
:1047E0000101CA33C933DF2AE8D789968994E55293
:1047F000E552E7CFD9FF1200D9CFE6FFE1CFD9FFCD
:10480000E652FE0EDB500101CB6FCC6BDF6A040E6B
:10481000DF5C15E289960000000000000101CB5129
:10482000010B02E0898401D0899489860000000090
:104830000000D8900101CC33CB33DF2AE8D789962A
:104840008994E552E552E7CFD9FF1200D9CFE6FFB0
:10485000E1CFD9FFE6528994DF6A040EDF5C0AE2F9
:10486000899600000000000089860000000000001A
:10487000DF2AF3D70C0EE66E1FEC2FF0E552899677
:10488000780EE66E49EC2FF0E552DF6A100EDF5C21
:104890000AE28986000000000000899600000000FE
:1048A0000000DF2AF3D7E552E552E7CFD9FF120027
:1048B000D9CFE6FFE1CFD9FFE6528994DF6A040E33
:1048C000DF5C0AE289960000000000008986000093
:1048D00000000000DF2AF3D789963C0EE66E08EC54
:1048E0002FF0E552DF6A100EDF5C0AE289860000D5
:1048F000000000008996000000000000DF2AF3D7C6
:10490000E552E552E7CFD9FF1200D9CFE6FFE1CF5C
:10491000D9FF020EE1268B808A94898AEFEC1FF082
:104920009296899692948994010EE66E08EC2FF087
:10493000E552DE6ADD6ADECF0BF0DDCF0CF0D890F9
:104940000C5004E6040E0B5C000E0C5813E28A8433
:10495000899A0C0EE66E49EC2FF0E5528A94898A0A
:10496000010EE66E08EC2FF0E552DF2A010E01E39E
:10497000DB2AE1D7B20EE66EBEEC20F0E552C20EA5
:10498000E66EBEEC20F0E552120EE66EBEEC20F0B4
:10499000E5520A0EE66EBEEC20F0E5528A84899A52
:1049A0001E0EE66E08EC2FF0E552F56E020EE15C8D
:1049B00002E2E16AE552E16EF550E552E7CFD9FF38
:1049C0001200ECEC1FF08A94898A0C0EE66E08EC5B
:1049D0002FF0E552899AA1EC2BF0928692848B906D
:1049E0001200050EE66E0E0EE66EE66A9FDEE552DA
:1049F000E552E552F60EE66E6E0EE66EE66A96DE5D
:104A0000E552E552E552E66A0E0EE66EE66A8EDE85
:104A1000E552E552E552F70EE66E6E0EE66EE66A78
:104A200085DEE552E552E5523C0EE66E0E0EE66E70
:104A3000E66A7CDEE552E552E552F80EE66E6E0E51
:104A4000E66EE66A73DEE552E552E552010EE66E69
:104A5000010EE66E0C0EE66E69DEE552E552E55299
:104A6000040EE66E0E0EE66EE66A60DEE552E55274
:104A7000E552F60EE66E6E0EE66EE66A57DEE5521B
:104A8000E552E552800EE66E800EE66E0C0EE66E86
:104A90004DDEE552E552E552E66AE66AE66A46DE32
:104AA000E552E552E55201D81200D9CFE6FFE1CF39
:104AB000D9FFE6528994DF6A040EDF5C0AE2899628
:104AC0000000000000008986000000000000DF2ACE
:104AD000F3D78996F00EE66E08EC2FF0E552F00E53
:104AE000E66E08EC2FF0E552DF6A100EDF5C0AE29A
:104AF0008986000000000000899600000000000088
:104B0000DF2AF3D7E552E552E7CFD9FF1200D9CF1C
:104B1000E6FFE1CFD9FF030EE126A60EE66E840E76
:104B2000E66EE66A03DEE552E552E552FC0EDBCFA7
:104B3000F3FFDB2AF350EA6A010FE96E010EEA2265
:104B4000EF50E66E0E0EE66EE66AF0DDE552E552D7
:104B5000E552F60EE66E6E0EE66EE66AE7DDE552AB
:104B6000E552E552FC0EDBCFF3FFDB2AF350EA6A95
:104B7000010FE96E010EEA22EF50E66E0E0EE66EB0
:104B8000E66AD4DDE552E552E552F70EE66E6E0EAA
:104B9000E66EE66ACBDDE552E552E552FC0EDBCF70
:104BA000F3FFDB2AF350EA6A010FE96E010EEA22F5
:104BB000EF50E66E0E0EE66EE66AB8DDE552E5529F
:104BC000E552F80EE66E6E0EE66EE66AAFDDE55271
:104BD000E552E552DF6A200EDF5C2DE2DF50E76E22
:104BE000FD0EDBCFE9FFFE0EDBCFEAFFE750E92643
:104BF000000EEA22020EEFCFDBFFDF28E76EFD0E8C
:104C0000DBCFE9FFFE0EDBCFEAFFE750E926000E1F
:104C1000EA22010EEFCFDBFF020EDBCFE6FF010E33
:104C2000DBCFE6FF0D0EE66E81DDE552E552E55283
:104C3000020EDF26D0D7DF6A0F0EDF5C28E2FC0E03
:104C4000DBCFF3FFDB2AF350EA6A010FE96E010EB6
:104C5000EA22020EEFCFDBFFFC0EDBCFF3FFDB2AF5
:104C6000F350EA6A010FE96E010EEA22010EEFCF5E
:104C7000DBFF020EDBCFE6FF010EDBCFE6FF0D0E02
:104C8000E66E54DDE552E552E552DF2AD5D7FC0E3B
:104C9000DBCFF3FFDB2AF350EA6A010FE96E010E66
:104CA000EA22020EEFCFDBFFFC0EDBCFF3FFDB2AA5
:104CB000F350EA6A010FE96E010EEA22010EEFCF0E
:104CC000DBFF020EDBCFE6FF010EDBCFE6FF0F0EB0
:104CD000E66E2CDDE552E552E5520CD8F56E030E7A
:104CE000E15C02E2E16AE552E16EF550E552E7CFA0
:104CF000D9FF1200D9CFE6FFE1CFD9FFE652899460
:104D0000DF6A040EDF5C0AE2899600000000000002
:104D10008986000000000000DF2AF3D70C0EE66E43
:104D200008EC2FF0E5528996000000000000DF6AD1
:104D3000100EDF5C0AE28986000000000000899600
:104D4000000000000000DF2AF3D7E552E552E7CF6C
:104D5000D9FF1200D9CFE6FFE1CFD9FF080EE12637
:104D6000040EDB6A050EDB6A060EDB6A070EDB6AE1
:104D7000FD0EDBCF06F0FE0EDBCF07F0020E06C005
:104D8000DBFF030E07C0DBFFDE6ADD6ADECF0BF060
:104D9000DDCF0CF0020EDBCF0DF0030EDBCF0EF0FB
:104DA0000D500B5C0E500C5824E284C1E6FF66ECFB
:104DB00020F0E5522BEC21F0F3CF0BF0F4CF0CF008
:104DC0000D6A0E6AD950040FE96EDACFEAFF0B5074
:104DD000EE260C50EE220D50EE220E50EE2286C131
:104DE000E6FF66EC20F0E552DF2A010E01E3DB2A44
:104DF000CDD7700EE66E66EC20F0E552030EE66E3F
:104E000008EC2FF0E552D950040FE96EDACFEAFF33
:104E1000EE52EE52EE6AEE6A040EDBCF0BF0050E98
:104E2000DBCF0CF00BC0F3FF0CC0F4FF00D0F56E2D
:104E3000080EE15C02E2E16AE552E16EF550E552EE
:104E4000E7CFD9FF1200D58E9298F28A1200D59E34
:104E5000F29A9288899812008150200B01E0010E8D
:104E60000101005D0AE08150200B01E0010E01010B
:104E7000006F81BA02D0010E02D0000E00D01200E5
:104E8000D9CFE6FFE1CFD9FF020EE126F56E020E83
:104E9000E15C02E2E16AE552E16EF550E552E7CFEE
:044EA000D9FF120024
:0C4EA4006C500BE1040100513C0BE84293
:104EB000E8420D0802E108D801D03ED804D0040E23
:104EC0006C5C01E14BD81200D9CFE6FFE1CFD9FFEE
:104ED000E6520101D76B0101D86B0101DD6BDE6B7E
:104EE000EAEC28F0DF6ADF500B6E0C6A010E0B5CF7
:104EF000000E0C581BE20101D85101E017D0F76AEF
:104F0000DF34FE0BF736F66E3C0EF6265D0EF7220A
:104F10000900F5CF0BF00800F5CF0CF004D00CC061
:104F2000FAFF0B50F96EFBDFDF2ADDD7F4D8E5522C
:104F3000E552E7CFD9FF1200020E0101D75D0CE167
:104F4000A6D8040100BD04D00401C80E006F03D030
:104F50000401880E006F01D02DD91200040E01014A
:104F6000E45D0CE112C46EFF6E50000804E2010122
:104F7000050EE46F03D00101030EE46F0101D705B4
:104F80000CE10DD8040104BD04D00401C80E046F67
:104F900003D00401880E046F01D00CD91200D9CFC0
:104FA000E6FFE1CFD9FF020EE1260101080EDD5D2B
:104FB000000EDE5905E2DDC1DEFFDEC1DDFF03D0FC
:104FC000080EDE6EDD6A0401049304010491010EF3
:104FD000DB5004010413DFCF05F4000EDB500101A8
:104FE000DD5F010EDB500101DE5B0101180EDB6F9E
:104FF000040EDC6F0101E5A320D0D9CFE9FFDACFA1
:10500000EAFFEE50ED1018E0D9C1F6FFDAC1F7FF64
:105010000800F550DBC1E9FFDCC1EAFFEF6E0101DA
:10502000DB2B000EDC230101D92B000EDA23DF0677
:10503000010E01E2DB06E1D71ED0D9CFE9FFDACFBE
:10504000EAFFEE50ED1017E0D9C1E9FFDAC1EAFF3F
:10505000EF50DBC1E9FFDCC1EAFFEF6E0101DB2BA2
:10506000000EDC230101D92B000EDA23DF06010E2E
:1050700001E2DB06E2D7F56E020EE15C02E2E16AD4
:10508000E552E16EF550E552E7CFD9FF1200D9CFD6
:10509000E6FFE1CFD9FF020EE126030E0401001561
:1050A000E76E010EE7CFDBFF01C4DFFFDE50010139
:1050B000DD27DD500101DE230101180ED96F040E3A
:1050C000DA6FD9CFE9FFDACFEAFFEE50ED1017E043
:1050D000D9C1E9FFDAC1EAFFEF50DBC1E9FFDCC16A
:1050E000EAFFEF6E0101DB2B000EDC230101D92B5F
:1050F000000EDA23DF06010E01E2DB06E2D7F56ED1
:10510000020EE15C02E2E16AE552E16EF550E55221
:10511000E7CFD9FF12006D980101D8510FE10401CA
:10512000080E016F0401100E026F040E036F0401DC
:10513000840E006F0401840E046F3BD0040110AF95
:1051400025D00101DD510401165D0101DE5104018C
:10515000175904E216C4DDF117C4DEF120DF0101A6
:10516000010ED76F0401080E016F0401100E026FCB
:10517000040E036F0401800E006F0401180E066F09
:10518000040E076F0401C80E046F13D00101020E54
:10519000D76F0401056B0401C80E046F0401080EEB
:1051A000016F0401180E026F040E036F0401C80E94
:1051B000006F12000101D76B0401080E016F04019A
:1051C000100E026F040E036F0401880E006F0401BD
:0451D000046B12005A
:0C51D40004011051600BE842E842E84280
:1051E000E842E842000901E058D004011151070AE1
:1051F00053E00B0A51E0070A42E0010A2CE00B0AD7
:1052000028E0020A26E0030A22E0080A12E0010A66
:105210000EE00F0A0AE0030A01E03ED00101010E90
:10522000D86F0101040EE46F38D038D836D093D847
:1052300034D00101010ED86F0101E60ED96F010EC5
:10524000DA6F0101E5930101010EDD6F26D0ABD8C5
:1052500024D0FAD822D00101010ED86F04011451D4
:105260000101D96FDA6BE70E0101D927010E0101A7
:10527000DA230101E5930101010EDD6F0ED001017A
:10528000010ED86F04011451EA6AE70FE96E010EAE
:10529000EA2212C4EFFF01D000D01200800E0401F8
:1052A000105D58E104011351030A34E0010A10E0D3
:1052B000030A01E04DD00101010ED86F0101EE0E8D
:1052C000D96F5B0EDA6F120E0101DD6FDE6B40D01D
:1052D0000101010ED86F04011251F66EF76AD890E1
:1052E000F636F7362E0EF6265D0EF7220900F5CFBC
:1052F000D9F10A00F5CFDAF1020E0101F76AD925DA
:10530000F66EDA51F7220900F5CFDDF10A00F5CF8C
:10531000DEF11ED00101010ED86F04011251F66EAC
:10532000F76AD890F636F736320EF6265D0EF7227B
:105330000900F5CFD9F10A00F5CFDAF1D9C1F6FFAE
:10534000DAC1F7FF0800F5500101DD6FDE6B00D018
:105350000101E58312000101010ED86F0F0EE66E08
:10536000710EE66E0F0EE66E2BEC2DF0E552E55257
:10537000E552010EE66EE70EE66E010EE66E2BECD0
:105380002DF0E552E552E55212C4E6F10401125146
:1053900004E10101050EE46F05D00101060EE46F82
:1053A00000EC2BF012000401186B0401196B0401CE
:1053B00010511F0B020A15E0030A0FE0010A01E079
:1053C00035D00101010ED86F02D00401188101010E
:1053D000E5A102D00401188329D00101010ED86F84
:1053E00025D00101010ED86F040114510F0B080DD7
:1053F000F3500C6A000F0B6E040E0C2204011451C2
:10540000800B01E0010E040DF35001010B24DB6F52
:10541000000E0C20DC6FDBC1E9FFDCC1EAFFEF50BE
:10542000040B03E00401010E186F00D00101D80540
:105430000AE10101180ED96F040EDA6F0101E5933C
:105440000101020EDD6F12000401120511E10401D9
:1054500010511F0B00090CE10101010ED86F030E62
:105460000401115D03E10101E58102D00101E59133
:10547000040112513EE1040110511F0B020839E1F1
:10548000040114510F0B000934E00101010ED86F23
:10549000040114510F0B080DF3500C6A000F0B6E32
:1054A000040E0C2204011451800B01E0010E040DC6
:1054B000F35001010B24DB6F000E0C20DC6F030E98
:1054C0000401115D07E1840EDBC1E9FFDCC1EAFFE5
:1054D000EF6E0FD0040114AF06D0DBC1E9FFDCC1D1
:1054E000EAFFEF6A06D0880EDBC1E9FFDCC1EAFF04
:0454F000EF6E120049
:0C54F400040110511F0B010801E07DD0E5
:105500000401145101E079D0060E0401115D2FE170
:1055100004011351230A28E0010A13E0030A01E001
:1055200024D00101020ED86F0101E60505E1010159
:10553000120ED96F5C0EDA6F090E0101DD6FDE6BA2
:1055400014D00101020ED86F0101E60505E1010149
:10555000110ED96F5D0EDA6F0101E60504E11D0E33
:105560000101DD6FDE6B01D000D00101E583040194
:105570001051600BE842E842E842E842E842010884
:1055800001E03BD0040111510B0A31E0080A21E08F
:10559000090A19E0080A09E00B0A05E0080A01E017
:1055A0002CD02CD82AD02BD828D00101020ED86FAD
:1055B0000101E80ED96F010EDA6F0101E5930101D7
:1055C000010EDD6F1AD00101020ED86F13C4E8F18D
:1055D00014D00101020ED86F0101E90ED96F010E3E
:1055E000DA6F0101E5930101010EDD6F06D00101C3
:1055F000020ED86F12C4E9F100D01200120012009E
:105600000101EA6B1E0E716E0401400E096F040168
:10561000200E0A6F040E0B6F0401880E086F040140
:10562000600E0E6F040E0F6F0401400E0C6F12001F
:10563000D9CFE6FFE1CFD9FFE652FC0EDB504008A0
:1056400005E2400EF36EFC0EF3CFDBFFDF6AFC0ECB
:10565000DB50DF5C19E2DF50E76EFD0EDBCFE9FFC8
:10566000FE0EDBCFEAFFE750E926000EEA22EF50FC
:10567000E66EDF50EA6A600FE96E040EEA22E55238
:10568000E750EF6EDF2AE3D7FC0EDBCF0DF4400EC0
:1056900004010C1704010C7D880E04010C13E55263
:1056A000E552E7CFD9FF1200D9CFE6FFE1CFD9FF0E
:1056B0000101EA6B040108BF39D0FC0EDBCF0BF00F
:1056C00004010951D8800B5403E2FC0E09C4DBFF2E
:1056D0000101EA6BFC0EDB500101EA5D1CE20101F5
:1056E000EA51EA6A200FE96E040EEA22EF50E66EF4
:1056F0000101EA51E76EFD0EDBCFE9FFFE0EDBCFC5
:10570000EAFFE750E926000EEA22E552E750EF6E85
:105710000101EA2BDFD70401400E096F400E04019E
:1057200008170401087D880E040108130101EA51DD
:0A57300000D0E552E7CFD9FF1200C8
:06573A008A940C0EBA6E09
:105740001200BA6A1200050EC26E3E0EC06E010152
:10575000DF6B0101E06B9E9C9D8CC2821200C26ACD
:105760009D9C1200CF6ACE6AB10ECD6E9E909D8038
:1057700012009D909E90CD6A8B9012008A888A9428
:10578000F1DF0101938712008A948A88EBDF01011F
:1057900093891200D8CFE4FFE0CFE4FFE46EDACFC4
:1057A000E4FFE2CFDAFFE9CFE4FFEACFE4FFF6CF90
:1057B000E4FFF7CFE4FFF5CFE4FFF3CFE4FFF4CF4E
:1057C000E4FFFACFE4FF00EE00F00B0EE80403E381
:1057D000EECFE4FFFBD700EE0BF0040EE80403E38A
:1057E000EECFE4FFFBD7E652D9CFE6FFE1CFD9FFFA
:1057F000E6529EAC4BD09E9C050EC25C19E18150D6
:10580000100B0DE101019851C45C09E2080E010181
:10581000DF5D02E1B3DF02D00101DF2B02D0010125
:10582000DF6BC4CF95F1C3CF94F1010EC26E2DD0C2
:10583000C2042BE10C0EBA6EBA500CE00101E25129
:10584000D880C45401E2BB6A0101E351C45C02E2A6
:10585000E1C1BBFF8150040B10E08050200B0DE133
:1058600001019951C45C09E2080E0101E05D02E109
:105870008BDF02D00101E02B02D00101E06BC4CF2D
:1058800097F1C3CF96F1050EC26EC282F2A406D084
:10589000F2948978F60ED76EBD0ED66E9E50010B2F
:1058A00005E09D50010B02E09E908B70E552E552A1
:1058B000E7CFD9FFE55200EE0EF0040EE80403E353
:1058C000E5CFEDFFFBD700EE0AF00B0EE80403E393
:1058D000E5CFEDFFFBD7E5CFFAFFE5CFF4FFE5CF4E
:1058E000F3FFE5CFF5FFE5CFF7FFE5CFF6FFE5CF17
:1058F000EAFFE5CFE9FFE5CFDAFFE550E5CFE0FFCE
:06590000E5CFD8FF100006
:0A5906006DA610D802D06DB614D8BB
:105910000101E40509E16DBA07D0686A696A698026
:1059200069880101020EE46F12006D6A696A6D8672
:105930000101010EE46F12006D6A696A0101E46BF6
:105940001200FADF12000101E45101E13AD068507F
:10595000040B04E06950040B01E038D86DB231D07B
:105960006850010B04E06950010B01E052D8685007
:10597000100B04E06950100B01E024D86850400B74
:1059800004E06950400B01E039D86850200B04E076
:105990006950200B01E034D86850020B04E06950D4
:1059A000020B01E034D8030E0101E45D01E209D0ED
:1059B0006850080B06E06950080B03E052EC27F032
:1059C00068961200698468986D8212006D926994DD
:1059D000689412000101E5A110D0F8DF6D84010187
:1059E000080EEB6F070EEC6F0101EB07000EEC5B8E
:1059F0000101EB51EC11F8E16D941200689C12006A
:105A000070A003D0DAEC28F07090689A12006892C7
:105A100012006A6A686A9F0E6B6E7B0E696E6E6A10
:105A20000F0EE66E710EE66E0F0EE66E14D8E5529E
:105A3000E552E552160E706E68A602D06896FCD745
:105A40006D98DAEC28F00101E5910101E66B0101A6
:105A5000030EE46F1200D9CFE6FFE1CFD9FFFD0EB0
:105A6000DBCFE9FFFE0EDBCFEAFFFC0EDB5004E0EC
:105A7000EE6AFC0EDB06F9D7E552E7CFD9FF12003C
:105A8000D9CFE6FFE1CFD9FF060EE12692868994B1
:105A9000929480A6FED78984020EDB6A030EDB6A2D
:105AA000020EDBCF0BF0030EDBCF0CF00D6AD890AB
:105AB0000D50000A06E6C80E0B5CAF0E0C58000E27
:105AC0000D5850E280B648D08994DE6ADD6ADECF98
:105AD0000BF0DDCF0CF0080E0B5C000E0C5821E231
:105AE00080A6FED7FE0EDBAE02D0898401D0899459
:105AF000040EDB6A050EDB6A80A606D0040EDB2AE4
:105B0000050E01E3DB2AF8D7FE0EDBCFF3FFF39E91
:105B1000F346FE0EF3CFDBFFDF2A010E01E3DB2AA3
:105B2000D6D780B6FED7DE6ADD6ADECF0BF0DDCFDA
:105B30000CF0040EDBCF0DF0050EDBCF0EF00D5098
:105B40000B5C0E500C5805E2DF2A010E01E3DB2A44
:105B5000ECD78994010E08D0020EDB2A030E01E374
:105B6000DB2A9ED7000E00D0F56E060EE15C02E245
:105B7000E16AE552E16EF550E552E7CFD9FF120038
:105B8000D9CFE6FFE1CFD9FF020EE12692868994B4
:105B9000929480A6FED7898480B6FED78994928499
:105BA000010EDB6A080EF36E010EDBCFF4FFF3503B
:105BB000F45C0DE280A6FED780B6FED7DF9EDF46FE
:105BC00080A402D0000EDB80010EDB2AEBD792947A
:105BD0008994DF5000D0F56E020EE15C02E2E16ACA
:0E5BE000E552E16EF550E552E7CFD9FF120015
:025BEE001201A2
:105BF000000200000008D804330001000102030283
:105C00000902290001010280320904000002030098
:105C10000000092101000001221D00070581034049
:105C200000010705010340000109022000010204F0
:105C300080320904000002FF0000000705810340D4
:105C40000001070501034000010403090434034D6A
:105C5000006900630072006F0063006800690070F3
:105C600000200054006500630068006E006F006C47
:105C7000006F0067007900200049006E0063002E6D
:105C80000048035000490043006B00690074002085
:105C900000320020004D006900630072006F006355
:105CA000006F006E00740072006F006C006C006585
:105CB0000072002000500072006F006700720061E7
:105CC000006D006D0065007200160350004900432E
:105CD0000031003800460032003500350030003217
:105CE000035000490043006B00690074002000323B
:105CF00000200043006F006E0066006900670075B9
:105D00000072006100740069006F006E00200032B4
:105D1000000600FF0901A10119012940150026FF15
:105D200000750895408102190129409102C0005C6C
:0E5D3000295C495C4D5C815CC95CDF5CF4540D
:025D3E002A0E2B
:105D4000F66E200EF76E000EF86E01010900F55098
:105D5000D26F0900F550D36F03E1D26701D03DD077
:105D60000900F550CD6F0900F550CE6F0900F550D0
:105D7000CF6F09000900F550E96E0900F550EA6E91
:105D8000090009000900F550D06F0900F550D16FE6
:105D900009000900F6CFD4F1F7CFD5F1F8CFD6F14D
:105DA000CDC1F6FFCEC1F7FFCFC1F8FF0101D0533F
:105DB00002E1D15307E00900F550EE6ED007F8E29A
:105DC000D107F9D7D4C1F6FFD5C1F7FFD6C1F8FF87
:0C5DD0000101D207000ED35BBFD7120008
:045DDC0005D813D8FB
:105DE000ACEC10F0FCD71200140E6F6E0101E46BE6
:105DF0000101E56B0101E66B689668966896689606
:105E000016EC10F0120083EC2CF0A3EC2CF0120036
:105E1000FF0EE350106EEF0E01D0F30EE76EE72E8B
:105E20000FEF2FF00C0E0F6EE76AE72E15EF2FF035
:0E5E30000F2E14EF2FF0102E0DEF2FF012009A
:025E3E00FF0E55
:105E4000E350106E480E01D04C0EE76EE72EFED7E1
:0E5E5000E76AE72EFED7102EF7D700001200EB
:025E5E00FF0E35
:105E6000E350106E1B0E00D001D0200EE76EE72E1F
:0A5E7000FED7102EFAD700D0120062
:065E7A0013EE00F023EE20
:105E800000F0F86A0A9C9FEC2EF0EEEC2EF0FDD7A5
:025E90001200FE
:0E5E9200FF0EE350E84E1200000000D000D0DA
:085EA00000D0E82EFAD7120031
:00000001FF
